:1000000082C0A6C0A0C3A4C02BC3A2C0A1C0A0C070
:100010009FC09EC09DC09CC09BC09AC099C0120149
:10002000010100000008C016DA27000101020001EA
:1000300005010902A1010901A1000509190129030E
:100040001500250195037501810295017505810152
:100050000501093009311581257F75089502810652
:10006000093895018106C0C000370038010101013F
:1000700001010102040810202803640069006700E0
:1000800069007300740075006D0070002E0063003D
:100090006F006D003A004D006F0075007300650041
:1000A000100344006900670069004B006500790097
:1000B0001C03640069006700690073007400750028
:1000C0006D0070002E0063006F006D0004030904D2
:1000D000090222000101008032090400000103002E
:1000E00000000921010100012238000705810308F1
:1000F000000A1201100100000008C016DA270001F2
:1001000001020301860511241FBECFE5D2E0DEBF48
:10011000CDBF10E0A0E6B0E0ECE5FBE002C005904A
:100120000D92A436B107D9F720E0A4E6B0E001C0F3
:100130001D92AC3BB207E1F710E0C3E8D0E003C08A
:100140002197FE01F6D4C238D107D1F75AD404C59D
:1001500057CFE3E7F0E09491EDE6F0E0E491EE2391
:1001600091F02AB52F7C2ABDF0E0E659FF4FA4910B
:10017000B0E0811109C08FB7F8942C91E92FE09578
:10018000E223EC938FBF08958FB7F894EC91E92B9D
:10019000F8CF2F923F924F925F926F927F928F9201
:1001A0009F92AF92BF92CF92DF92EF92FF920F9306
:1001B0001F93CF93DF9300D000D0CDB7DEB74B01B4
:1001C0005C012FB7F8948091850090918600A091F2
:1001D0008700B09188002FBF2FB7F894C09085009A
:1001E000D0908600E0908700F09088002FBF8C1997
:1001F0009D09AE09BF091C012D01280C391C4A1CA0
:100200005B1C520141018091A300835087FD3CC0DB
:100210009091A1009D32B1F58830A1F58091A200A6
:10022000ECE0F0E0E81BF109EA55FF4F83EC809326
:1002300089008AE580936100109274002081207605
:1002400009F465C189E690E090937600809375008B
:10025000203209F05AC1818124E0813051F082308E
:1002600009F04EC122E630E030937600209375000D
:1002700021E08781811104C08681821708F4282F2C
:10028000209360001092A3008091610084FF42C01F
:10029000809160008F3F09F43DC08983893010F060
:1002A00098E09983982F2981921B909360009091F8
:1002B000890028E89227909389008823E1F08091B3
:1002C0007500909176002091740026FFABC1AAE8DA
:1002D000B0E0FC01298134913D9331962150D9F74A
:1002E0002981215030E02F5F3F4F820F931F909361
:1002F00076008093750069818AE890E00DD299813B
:100300009C5F99839C3019F08FEF80936000398156
:100310003093610084E196B3987131F48150D9F73C
:100320001092A4001092A000662463948111612CA5
:1003300090917700691699F1882379F1F89488E013
:1003400090E09C838B83712C90E899832981270D01
:100350002A8321BFE5D18C01843399400CF47A8043
:100360008981869589832B813C81215031093C8389
:100370002B83232B59F78FEF870D81BF872D90E0BB
:1003800001969C838B8381B72B813C818217130656
:1003900009F00CF450C171BE7894609277008FB769
:1003A000F89400918500109186002091870030918B
:1003B00088008FBF4091810050918200609183003E
:1003C000709184008091620090E0880F991F880FDF
:1003D000991F092E000CAA0BBB0B041B150B260B37
:1003E000370B081719072A073B0778F0840F951F6A
:1003F000A61FB71F8093810090938200A093830073
:10040000B093840031E03093800044E050E068E72E
:1004100070E08CE790E093D3892B19F081E0809312
:10042000800080918000882309F44BC08091940063
:1004300084FF47C01092800080917C0090917D00E5
:10044000A0917E00B0917F008093690090936A0034
:10045000A0936B00B0936C00809378009093790028
:10046000A0937A00B0937B0010927D0010927E00E2
:1004700010927F001092790010927A0010927B0007
:100480008091940084FFE8C08091950098E88927C6
:1004900080939500809169008093960080916A0016
:1004A0008093970080916B008093980080916C00FE
:1004B0008093990064E086E990E02ED188E08093F3
:1004C0009400D701C60112141304140415040CF48B
:1004D00083CE0F900F900F900F90DF91CF911F91CF
:1004E0000F91FF90EF90DF90CF90BF90AF909F90D3
:1004F0008F907F906F905F904F903F902F900895D6
:100500008A3019F483818093620020E0B2CE928118
:1005100010929200818181110AC01092930082E9A9
:1005200090E022E09093760080937500A2CE853013
:1005300029F49093A40082E990E0F4CF863009F08A
:100540005AC08381813059F482EF90E09093760015
:100550008093750022E180E4809374008ACE82301B
:1005600041F420ED30E0309376002093750022E2D4
:10057000F2CF833041F5911108C08CEC90E090935C
:1005800076008093750024E0E6CF913041F420EBB3
:1005900030E030937600209375002CE1DCCF923070
:1005A00041F480EA90E0909376008093750020E11A
:1005B000D2CF933081F628E730E030937600209355
:1005C000750028E2C8CF813241F482EE90E090932A
:1005D00076008093750029E0BECF823209F0BBCF50
:1005E00080917100909172009093760080937500D5
:1005F00020917000B0CF883071F0893019F4909359
:10060000730099CF8A3059F08B3009F094CF8BE486
:100610008093950090CF83E790E021E083CF82E93B
:1006200090E0FBCFDC01EAE8F0E029813D913193D5
:100630002150E1F755CE74D08453994097FF03C001
:100640009195819591098017910714F471B68C01E9
:1006500081B78F5F81BF97CE8AE5809394001ACFD0
:1006600078941F920F920FB60F9211242F933F93FD
:100670008F939F93AF93BF93809185009091860055
:10068000A0918700B0918800309168002CE7230F7B
:100690002D3728F02FEF230F0196A11DB11D2093B8
:1006A00068008093850090938600A0938700B093A4
:1006B00088008091640090916500A0916600B091DF
:1006C00067000196A11DB11D8093640090936500A1
:1006D000A0936600B0936700BF91AF919F918F91F7
:1006E0003F912F910F900FBE0F901F901895A82F3C
:1006F000B92F80E090E041E050EA609530E009C019
:100700002D9182279795879510F084279527305E45
:10071000C8F36F5FA8F30895EADF8D939D93089562
:10072000A6E088279927AA9569F00197E1F3B39984
:10073000FCCFB39BFECF81E09927A6B3019611F0C1
:10074000A871D9F70895CF93CFB7CF93C395B39B33
:10075000E9F7B39B0BC0B39B09C0B39B07C0B39B26
:1007600005C0B39B03C0B39B01C0D5C00F92DF93FC
:10077000C091A200DD27CA55DF4F012EB39B03C0F5
:10078000DF910F90E6CF2F930F931F934F932FEF8F
:100790004F6F06B303FB20F95F933F9350E03BE0BC
:1007A00065C016B30126502953FDC89556B30127DD
:1007B00003FB25F92F7306B3B1F05027102713FB65
:1007C00026F906B22230F0F000C016B3012703FB71
:1007D00027F90126502906B22430E8F54F77206822
:1007E00016B30000F6CF50274F7D206206B2102FBF
:1007F000000000C006B300265029102713FB26F97D
:1008000006B2E2CF4F7B06B3206400C0DACF0126E8
:100810005029187106B269F14E7F2160012F16B37D
:1008200028C0002650294D7F06B22260102F29C013
:10083000012650294B7F06B22460012F2DC016B32C
:1008400001265029477F2860000006B22EC04F7E47
:1008500006B3206130C0422706B3499300265029D1
:10086000102706B24FEF13FB20F9297F16B379F258
:10087000187159F10126502906B2012703FB21F90D
:10088000237F06B371F2002650293150D0F006B212
:10089000102713FB22F9277E16B351F201265029A7
:1008A000012703FB06B223F92F7C49F2000006B3AF
:1008B000102713FB24F90026502906B22F7939F2AC
:1008C00070CF10E21ABF002719C03B503195C31BEF
:1008D000D04010E21ABF0881033C09F10B34F9F053
:1008E0002091A0001981110F1213EDCF4A81441FEE
:1008F000093651F10D3211F0013E29F70093A500A0
:100900003F915F914F911F910F912F91DF910F9028
:10091000CAB7C5FD1BCFCF91CFBFCF9118952091FE
:10092000A500222369F31091A300112379F5343037
:100930007AF13093A3002093A1001091A2003BE034
:10094000311B3093A20024C00091A3000130F4F4C5
:100950000AE54F7049F43091610034FD1AC00093EC
:100960006100C9E8D0E019C03091940034FD11C095
:1009700000939400C5E9D0E010C0052710E000C046
:1009800021C0052710E0C89508BB14C03AE501C096
:1009900032ED032EC0E0D0E032E017B31861C39A05
:1009A00008B317BB58E120E84FEF20FF052708BB2D
:1009B000279517951C3F28F700004552B0F720FFF8
:1009C0000527279508BB17951C3FB8F629913A953E
:1009D00061F7077E1091A400110F08BBC250D040F0
:1009E00011F01093A00010E21ABF086017B3177E31
:1009F000402F477E54E05A95F1F708BB17BB48BB20
:100A00007FCF789480B7806880BF80B7806480BFD4
:100A10008CB580648CBD8FEF8DBD80B7807F876083
:100A200080BF89B7846089BF83B7887F83BF8AB559
:100A30008C7F81608ABD83B7877F83BF83B7887FC0
:100A4000836083BF86B1876086B9379AF894BB9A72
:100A50002FE182E19AE0215080409040E1F700C010
:100A60000000BB98AC9A8BB780628BBF8BE48093FD
:100A700095008AE58093940078942FB7F89480913C
:100A8000850090918600A0918700B09188002FBFCB
:100A90008093810090938200A0938300B0938400A0
:100AA000E3E7F0E02491EDE6F0E0E491EE2389F055
:100AB0008E2F90E0FC01E859FF4FA491B0E08659D9
:100AC0009F4FFC0184918FB7F894EC91E22BEC934B
:100AD0008FBFD2E0CEEF81E03CDBD0937D0010925F
:100AE0007E0010927F0062E370E080E090E051DBD6
:100AF000C0937D0010927E0010927F0080E029DB81
:100B000060E375E780E090E044DBE5CF80E390E0D0
:100B1000909372008093710088E3809370008EE15F
:100B200090E090936F0080936E0082E180936D005F
:100B30000895EE0FFF1F0590F491E02D0994FB013D
:100B4000DC0104C08D910190801921F44150504086
:0C0B5000C8F7881B990B0895F894FFCF9C
:040B5C00FF5A050037
:00000001FF
